:100000000C9484000C94A5000C94A5000C94A500FD
:100010000C94A5000C94A5000C94A5000C94A500CC
:100020000C94A5000C94A5000C94A5000C94A500BC
:100030000C94A5000C94A5000C94A5000C94A500AC
:100040000C94A5000C94DF020C94A5000C94A50060
:100050000C94A5000C94A5000C94A5000C94A5008C
:100060000C94A5000C9400010C94A5000C94A50020
:100070000C94A5000C94A5000C94A5000C94A5006C
:100080000C94A5000C94A5000C94A5000C94A5005C
:100090000C94A5000C94A5000C94A5000C94A5004C
:1000A0000C94A5000C94A5000C94A5000C94A5003C
:1000B0000C94A5000C94A5000C94A5000C94A5002C
:1000C0000C94A5000C94A5000C94A5000C94A5001C
:1000D0000C94A5000C94A5000C94A5000C94A5000C
:1000E0000C94A5000C9488010C94AF000C94BF00F4
:1000F0000C94ED000C94A7000C94DF000C94B70056
:100100000C94CA000C94D50011241FBECFEFD1E28D
:10011000DEBFCDBF00E00CBF13E0A0E0B2E0ECE436
:10012000F2E100E00BBF02C007900D92AE30B107C4
:10013000D9F72AE0AEE0B3E001C01D92A933B207BF
:10014000E1F70E9434040C9424090C940000E0911F
:100150001F03F091200380810E945C01F8CFE091A1
:10016000ED07F091EE0780810E945C01F8CFE091ED
:100170001508F091160880810E945C01F8CF0E945A
:1001800069018823E1F3E0911F03F091200381507E
:100190008083F5CF0E9469018823E1F3E091ED07A8
:1001A000F091EE078F5F8083F5CF0E94690188236D
:1001B000E1F3E0911508F09116088083F6CF2FEF58
:1001C00083E294EF215080409040E1F700C00000AE
:1001D00084E192E00E943A06F2CF8A3049F0909191
:1001E000C00095FFFCCF8093C60080E090E00895AA
:1001F0009091C00095FFFCCF9DE09093C600EFCF9B
:100200001F920F920FB60F9211240BB60F922F93DD
:100210003F934F935F936F937F938F939F93AF938E
:10022000BF93EF93FF938091C60080932A0A82E0E8
:1002300090E00E946403FF91EF91BF91AF919F9175
:100240008F917F916F915F914F913F912F910F907F
:100250000BBE0F900FBE0F901F9018959093C50086
:100260008093C40086E08093C20088E98093C10037
:1002700008959091C00095FFFCCF8093C60008952B
:100280008091C00087FFFCCF8091C60008958091C7
:10029000C000881F8827881F0895FC012081222321
:1002A00051F031969091C00095FFFCCF2093C6008D
:1002B00021912111F7CF08959091C00095FD06C0BE
:1002C0008091C00083E090E00C9464038093C600AA
:1002D000089580912A0A811106C081E090E00E9471
:1002E000640380912A0A10922A0A089580E092E01D
:1002F0009093360A8093350A1092C50082E380936A
:10030000C40086E08093C20088E98093C10008950C
:100310007894A0912B0AB0912C0A109789F012962C
:10032000ED91FC911397309759F014966D917D9152
:100330008D919C9117971995A0912B0AB0912C0A39
:1003400081E052968C9308950F931F93FC01538381
:10035000428304831583268337831386128611868E
:10036000108682E0828B88E891E0DB018C93119704
:100370009C9311971C9211971C9211971C921197A4
:100380001C9211971C9211971C9211971C92119715
:100390001C9211971C9211971C9211971C92119705
:1003A0001C9211971C9211971C9211971C921197F5
:1003B0001C9211971C9211971C9211971C921197E5
:1003C0001C9211971C9267517109718360831F9170
:1003D0000F910895CF93DF93FC01A081B181109715
:1003E000B1F084818130B9F01896CD91DC911997E4
:1003F000D183C083DB87CA87848181508483199627
:100400001C921E9218971B961C921E921A97CD0151
:10041000DF91CF9108951382128211821082EDCF65
:10042000DB011A962D913C911B97232B11F08FEF36
:10043000089518962D913C911997232BC1F7FC0133
:100440002481211115C071836083738362831B969D
:100450007C936E931A9719961C921E921897DC0142
:1004600014962C9114972F5F14962C9380E0089586
:100470000280F381E02D71876087DB011B96FC937E
:10048000EE931A9719961C921E921897FC0173838B
:100490006283E5CF0F931F93CF93DF93FC01C0815D
:1004A000D1818BE292E00E943A062097E9F00FE3B7
:1004B00012E089858F9388858F938B858F938A85AA
:1004C0008F93DF93CF931F930F930E94200608848E
:1004D000D985C02DEDB7FEB738960FB6F894FEBF9C
:1004E0000FBEEDBF209729F786E392E0DF91CF9111
:1004F0001F910F910C943A062F923F924F925F9268
:100500006F927F928F929F92AF92BF92CF92DF9223
:10051000EF92FF920F931F93CF93DF930BB60F923F
:100520000CB60F920DB71EB7C82FD92F08831983A9
:10053000C62FD72F088119810DBF1EBF0F900CB693
:100540000F900BB6DF91CF911F910F91FF90EF901D
:10055000DF90CF90BF90AF909F908F907F906F90E3
:100560005F904F903F902F900895C82FD92F08810A
:1005700019810DBF1EBF0F900CB60F900BB6DF9107
:10058000CF911F910F91FF90EF90DF90CF90BF9090
:10059000AF909F908F907F906F905F904F903F9023
:1005A0002F90189584E294EF9093890080938800AF
:1005B00082E080936F008CE08093810008951F9209
:1005C0000F920FB60F9211240BB60F922F933F93F9
:1005D0004F935F936F937F938F939F93AF93BF934B
:1005E000EF93FF930E94C303FF91EF91BF91AF91EF
:1005F0009F918F917F916F915F914F913F912F913B
:100600000F900BBE0F900FBE0F901F901895F8948F
:10061000EAE6F0E080818C608083ED9A6D9A7894B0
:100620000895CF93DF93F8948FE090E00E94FA044E
:10063000EC0190932E0A80932D0A83E190E00E94B2
:10064000FA0490932C0A80932B0A85E0E8E1F3E00A
:10065000DE0101900D928A95E1F785E0E3E1F3E098
:10066000DE01159601900D928A95E1F785E0EEE0A6
:10067000F3E0DE011A9601900D928A95E1F7CE0122
:100680000A960E94EA01BC0190932C0A80932B0ADF
:1006900080912D0A90912E0A0A960E941002E091F4
:1006A0002B0AF0912C0A128AEF2B61F00E94D202E1
:1006B0000E94070380912B0A90912C0ADF91CF9121
:1006C0000C94B5020E941B06CF93DF93C0912B0AB6
:1006D000D0912C0A8330910501F18130910509F404
:1006E00043C0029719F0DF91CF91089582E08A8B81
:1006F00080912D0A90912E0A0E94EA0190932C0A73
:1007000080932B0AFC01128AC817D90761F3BC0138
:10071000CE01DF91CF910C947C0283E08A8B809193
:100720002D0A90912E0ABE0105960E94100280911A
:100730002D0A90912E0A0A960E94EA01BC0190931C
:100740002C0A80932B0A80912D0A90912E0A0A96EA
:100750000E94100260912B0A70912C0AFB01128AF0
:10076000C617D707A9F6BFCF83E08A8BBE01809159
:100770002D0A90912E0A0E94100280912D0A9091CC
:100780002E0A0596B9CF80911D0390911E03019604
:1007900090931E0380931D036FE070E00E94D204CB
:1007A000892B09F0089588EB92E00E943A0687E5CC
:1007B00092E00E943A0680912D0A90912E0A0E94A2
:1007C0004A028AE090E00E9434068DE792E00E949F
:1007D0003A0680912D0A90912E0A05960E944A02AF
:1007E0008AE090E00E94340680912C0A8F938091D9
:1007F0002B0A8F9385EA92E09F938F930E942006A5
:100800008AE090E00E9434068AEB92E00E943A0669
:1008100080911508909116080E943A0685ED92E0A5
:100820000E943A068091ED079091EE070E943A06E9
:1008300080EF92E00E943A06809120038F9380918E
:100840001F038F938BE093E09F938F930E9420066A
:100850008DB79EB708960FB6F8949EBF0FBE8DBF9A
:1008600088EB92E00C943A060F931F930E94760156
:1008700082E090E00E94FA04909316088093150895
:1008800082E090E00E94FA049093EE078093ED07D7
:1008900082E090E00E94FA049093200380931F036B
:1008A00000E010E0980147EA50E060E275E08FEE6A
:1008B00097E00E94A40100E010E098014FEA50E0A8
:1008C00069E27AE087E199E00E94A40100E010E08B
:1008D000980147EB50E069ED76E08AED97E00E94E1
:1008E000A40100E010E098014FEB50E069ED77E0E3
:1008F00082E098E00E94A40100E010E098014AEC38
:1009000050E066E179E081E295E00E94A40100E018
:1009100010E0980145ED50E060E274E084E395E07A
:100920000E94A40100E010E098014FED50E069ED55
:1009300075E087E495E00E94A40164E375E088E136
:1009400093E00E94100261E275E088E193E00E946A
:10095000100262E078E088E193E00E9410026AED04
:1009600077E083E193E00E94100267E179E083E1A0
:1009700093E00E9410026FEE77E083E193E00E9423
:10098000100267E475E08EE093E00E94100281E2BD
:1009900092E00E943A060E94110380E090E01F91CD
:1009A0000F91089597FB072E16F4009407D077FD5A
:1009B00009D00E94E60407FC05D03EF4909581958D
:1009C0009F4F0895709561957F4F0895AA1BBB1B9B
:1009D00051E107C0AA1FBB1FA617B70710F0A61B3F
:1009E000B70B881F991F5A95A9F780959095BC0160
:1009F000CD0108950F931F93CF93DF93823091051C
:100A000010F482E090E0E091310AF091320A20E0A7
:100A100030E0A0E0B0E0309719F1408151810281CF
:100A2000138148175907C8F08417950769F4109780
:100A300031F012960C93129713961C9327C00093D3
:100A4000310A1093320A22C02115310519F04217DC
:100A5000530718F49A01BD01EF01DF01F801DBCF64
:100A600021153105F9F0281B390B2430310580F4AC
:100A70008A819B816115710521F0FB01938382833B
:100A800004C09093320A8093310AFE01329644C02A
:100A9000FE01E20FF31F81939193225031093983B4
:100AA00028833AC020912F0A3091300A232B41F439
:100AB00020911002309111023093300A20932F0AB6
:100AC00020910E0230910F022115310541F42DB70E
:100AD0003EB74091120250911302241B350BE09156
:100AE0002F0AF091300AE217F307A0F42E1B3F0BF8
:100AF0002817390778F0AC014E5F5F4F2417350790
:100B000048F04E0F5F1F5093300A40932F0A819395
:100B1000919302C0E0E0F0E0CF01DF91CF911F910F
:100B20000F910895CF93DF93009709F481C0FC01E2
:100B3000329713821282A091310AB091320A109733
:100B400081F420813181820F931F20912F0A3091EF
:100B5000300A2817390751F5F093300AE0932F0A2D
:100B600067C0ED0120E030E0CE17DF0740F44A8196
:100B70005B819E0141155105F1F0EA01F5CFD38368
:100B8000C28340815181840F951FC817D90759F43A
:100B900088819981840F951F0296918380838A8131
:100BA0009B81938382832115310529F4F093320AC6
:100BB000E093310A3DC0E901FB83EA8349915991F1
:100BC000C40FD51FEC17FD0761F480819181840F5C
:100BD000951F0296E90199838883828193819B8383
:100BE0008A83E0E0F0E012968D919C911397009734
:100BF00019F0FD01DC01F7CF8D919C9111979D01BA
:100C00002E5F3F4F820F931F20912F0A3091300AA1
:100C10002817390769F4309729F41092320A109294
:100C2000310A02C013821282B093300AA0932F0AB5
:100C3000DF91CF91089581E090E0F8940C9424091D
:100C4000CF93DF93CDB7DEB7AE014A5F5F4FFA01B6
:100C500061917191AF018091350A9091360A0E949D
:100C60006A06DF91CF9108956091350A7091360A36
:100C70000C948A080F931F93CF93DF93E091350A6A
:100C8000F091360A238121FF1BC08C01D0E0C0E027
:100C9000F80181918F016091350A7091360ADB016C
:100CA0001896ED91FC911997882331F01995892BAD
:100CB00079F3DFEFCFEFECCF8AE01995892B19F0AC
:100CC0008FEF9FEF02C08D2F9C2FDF91CF911F914F
:100CD0000F9108952F923F924F925F926F927F9261
:100CE0008F929F92AF92BF92CF92DF92EF92FF923C
:100CF0000F931F93CF93DF93CDB7DEB72B970FB62C
:100D0000F894DEBF0FBECDBF6C017B018A01FC01F0
:100D100017821682838181FFCCC1CE0101963C01EE
:100D2000F6019381F70193FD859193FF81917F01F6
:100D3000882309F4BAC1853239F493FD859193FF74
:100D400081917F01853229F4B60190E00E948A08E2
:100D5000E7CF912C212C312CFFE1F315D8F08B3209
:100D600079F038F4803279F08332A1F4232D2061B8
:100D70001DC08D3261F0803369F4232D216016C0CF
:100D8000832D8260382EE32DE4603E2E2AC0F32DA1
:100D9000F8601DC037FC2DC020ED280F2A3040F030
:100DA0008E32B9F436FC81C1232D2064322E19C055
:100DB00036FE06C08AE0989E200D1124922E11C0A6
:100DC000EAE02E9E200D1124222EF32DF0623F2EFC
:100DD00008C08C3621F4832D8068382E02C08836F6
:100DE00041F4F70193FD859193FF81917F0181117A
:100DF000B3CF982F9F7D9554933028F40C5F1F4FED
:100E00009FE399830DC0833631F0833771F08335CA
:100E100009F059C021C0F801808189830E5F1F4FFE
:100E200088248394912C530113C02801F2E04F0EC3
:100E3000511CF801A080B18036FE03C0692D70E01E
:100E400002C06FEF7FEFC5010E947F084C01820155
:100E5000F32DFF773F2E16C0280122E0420E511CD1
:100E6000F801A080B18036FE03C0692D70E002C099
:100E70006FEF7FEFC5010E9474084C01F32DF068FD
:100E80003F2E820133FC1BC0822D90E0881699060C
:100E9000B0F4B60180E290E00E948A082A94F4CF70
:100EA000F50137FC859137FE81915F01B60190E035
:100EB0000E948A0821102A9421E0821A9108811444
:100EC000910471F7E8C0843611F0893641F5F801D4
:100ED00037FE07C060817181828193810C5F1F4F53
:100EE00008C060817181072E000C880B990B0E5F82
:100EF0001F4FF32DFF763F2E97FF09C090958095E9
:100F0000709561957F4F8F4F9F4FF0683F2E2AE07D
:100F100030E0A3010E94C608882E861845C0853798
:100F200031F4232D2F7EB22E2AE030E025C0932D00
:100F3000997FB92E8F36C1F018F4883579F0B5C095
:100F4000803719F0883721F0B0C0E92FE061BE2E5C
:100F5000B4FE0DC0FB2DF460BF2E09C034FE0AC0E4
:100F6000292F2660B22E06C028E030E005C020E11F
:100F700030E002C020E132E0F801B7FE07C0608136
:100F80007181828193810C5F1F4F06C060817181E6
:100F900080E090E00E5F1F4FA3010E94C608882EDC
:100FA0008618FB2DFF773F2E36FE0DC0232D2E7F9A
:100FB000A22E891458F434FE0BC032FC09C0832DD4
:100FC0008E7EA82E05C0B82CA32C03C0B82C01C05F
:100FD000B92CA4FE0FC0FE01E80DF11D8081803305
:100FE00021F49A2D997EA92E09C0A2FE06C0B394C1
:100FF000B39404C08A2D867809F0B394A3FC11C081
:10100000A0FE06C0B21488F4280C922C9B180EC0C7
:10101000B21460F4B60180E290E00E948A08B394B2
:10102000F7CFB21418F42B1802C0982C212CA4FE70
:1010300010C0B60180E390E00E948A08A2FE17C0AB
:10104000A1FC03C088E790E002C088E590E0B6010B
:101050000CC08A2D867859F0A1FE02C08BE201C037
:1010600080E2A7FC8DE2B60190E00E948A08891414
:1010700038F4B60180E390E00E948A089A94F7CF92
:101080008A94F301E80DF11D8081B60190E00E9481
:101090008A088110F5CF222009F442CEB60180E201
:1010A00090E00E948A082A94F6CFF6018681978103
:1010B00002C08FEF9FEF2B960FB6F894DEBF0FBEE6
:1010C000CDBFDF91CF911F910F91FF90EF90DF90F7
:1010D000CF90BF90AF909F908F907F906F905F90D8
:1010E0004F903F902F900895FC0105906150704003
:1010F0000110D8F7809590958E0F9F1F0895FC01E1
:101100006150704001900110D8F7809590958E0F36
:101110009F1F08950F931F93CF93DF93FB012381AC
:1011200021FD03C08FEF9FEF2CC022FF16C0468128
:101130005781248135814217530744F4A081B1813E
:101140009D012F5F3F4F318320838C932681378110
:101150002F5F3F4F3783268314C08B01EC01FB01C7
:101160000084F185E02D1995892BE1F6D8011696BA
:101170008D919C911797019617969C938E93169735
:10118000CE01DF91CF911F910F910895FA01AA2707
:10119000283051F1203181F1E8946F936E7F6E5FBA
:1011A0007F4F8F4F9F4FAF4FB1E03ED0B4E03CD068
:1011B000670F781F891F9A1FA11D680F791F8A1F4B
:1011C000911DA11D6A0F711D811D911DA11D20D0B2
:1011D00009F468943F912AE0269F11243019305D6C
:1011E0003193DEF6CF010895462F4770405D41935D
:1011F000B3E00FD0C9F7F6CF462F4F70405D4A33AA
:1012000018F0495D31FD4052419302D0A9F7EACF71
:10121000B4E0A6959795879577956795BA95C9F7A0
:1012200000976105710508959B01AC010A2E069493
:101230005795479537952795BA95C9F7620F731F4C
:0C124000841F951FA01D0895F894FFCF97
:10124C000000000200000000ED00000000000000A3
:10125C00390A20000A736C656570696E672E2E2E34
:10126C00000A7374617274696E67007374617274CE
:10127C002D6C69737400656E642D6C697374005BFE
:10128C00633A2025702C20703A2025702C206E3A61
:10129C002025705D0A200052454144592051554586
:1012AC005545206465692070726F6365737369209E
:1012BC006469206C6574747572613A200052454102
:1012CC004459205155455545206465692070726F0D
:1012DC0063657373692064692073637269747475D0
:1012EC0072613A200043555252454E542050524F91
:1012FC00434553533A2025700A0053746174757337
:10130C002045786368616E67652042756666657214
:10131C0020313A20005374617475732045786368EA
:10132C00616E67652042756666657220323A2000F0
:10133C005374617475732045786368616E676520BA
:0E134C0042756666657220333A2000257300F4
:00000001FF
